:100000000C9453050C9470050C9470050C947005B9
:100010000C9470050C9470050C9470050C9470058C
:100020000C9470050C9470050C9470050C9470057C
:100030000C9470050C9470050C9470050C9470056C
:100040000C9470050C9470050C9470050C9470055C
:100050000C9470050C9470050C9470050C9470054C
:100060000C948B080C9470050A14BB15DA15F61560
:10007000561527164316801637149F16705103869F
:10008000400D4FEB3ECCD18735BDF50B5ED0F8F27D
:10009000D5E26C310CADFC21C378C106C24C55E6EB
:1000A0004A3448111EDAE71A84A096A7E37FAF63AB
:1000B0009CFA235B79C89EBAB2C922124BB3A1B68F
:1000C0003249A2E189391066C5078F54EA91CA3FC7
:1000D000F919F0D746BC281B61E82F6AAE9DF64E91
:1000E0000914774DDB1F2E7B7CF143A300B8138CE2
:1000F00085B9297588FDD2561C509741E53B60B5FE
:10010000C064EE98D62D25A4AACD7DA883C6ABBE2B
:100110004499263CCE9FBFD3CB767A7E82018A9AC1
:10012000801D0EB05CD43862F430E08E53B70257B5
:10013000ACA6520A6D9265172433457274B1B4F7B8
:100140005DED2CFF47375A90BBDF2A165995D9C46D
:10015000276773C768FEA5DD6B5F93D8EC053A8D02
:100160006EFB3DA96936F394DEEF156F8B9B080F8C
:10017000DC81182004E471CFE92B425801A0A96268
:10018000D63F85A7B6D4FA15661709BD5D14342687
:1001900059729154064FF8B05B7493998CF245CD27
:1001A000EA4EAD104AE5CAEEDFC66F9F888E02CCDC
:1001B00008A877946D21B128E43979966071811689
:1001C0002EE678B9C4469A42AEB77C43B3221A866B
:1001D000C2323D2D9CD229E9639BD131385E1E3657
:1001E00041BB03182B3EBF6861FC52C0DEE00A58D9
:1001F000135A00BE1C900E5312FDE26EBACE242795
:10020000447F87A3A1D55040E3F983F7C7A235C83F
:10021000DB19AB2F1125ED339E55E148AF7384DA1E
:100220002AAA51EB9D95B2CBE77080FE4C6504EF96
:10023000C5F1C33AB4F55F2389DD30A58BD3F6DC75
:100240004D64D7F08FEC56375CA40D07768A2C0BE3
:10025000B5D8C11FE83BF44B1B476C49677B92CF75
:10026000757E20D97D3C977AD0056B0F1DFB829857
:10027000578DF36ABCACC9A6FFB8690C4C4D720728
:100280005A49338DA2AB463D630DA097FFF0F5FAB6
:10029000C0E9DB62E4E17443DC86182937F406E246
:1002A000ED6F90481E2D1DEA739454DF25F6472705
:1002B000D91177C9841C5B5C5181A6223E2496C863
:1002C0008AEC827C09B8454A57BB2F50758E617005
:1002D0008C6CAFD0FDB41BAEDEFE3BB536BD550118
:1002E0000E9C41565FB3260383BA134BCAC50AF866
:1002F00060A5B9C7C39832FB12F9A792AA68F37830
:100300007E05202102E8BFF2B0598FD2CB87651558
:10031000F11AB230ADEE58A38B661F2CD75D19854C
:10032000A8E6D36BA10C91936A5E0B79E3DD004FD5
:100330003C896E7169A9AC40E59928C6314E7ACDE9
:10034000089E7DEF17FC88D8A46D4495D1B7D49B47
:10035000BE2A34642BCF2EEB38CE23E03A3FF77B16
:100360009F1053BC526716E7807604C4B6C1C27FA3
:100370009ADAD53942149DB10F35D6CCB9DA380C9A
:10038000A29C091F06B1B6FD1A692330C4DE01D153
:10039000F45829371C7DD5BFFFBDC8C9CF65BE7BCA
:1003A0007897986708B32657F7FA40AD8E75A67C04
:1003B000DB918B5199D4177A908DCE63CB4EA0AB45
:1003C000183A5B507F2174C1BBB8B7BA0B35953171
:1003D000599A4D04071E5A7613F37183D08603A8E9
:1003E0003942AA28E6E4D85DD3D06E6F96FB5EBC96
:1003F00056C25F859BE7AFD23B846AA753C5444989
:10040000A5F936723D2CD91BA1F54F939D68474144
:1004100016CA2A4CA387D6E5192E77156D70C0DF52
:10042000B20046EDC66C4360922DA922458F34552B
:10043000AEA40A6632E0DC02ACE8208C89624AFE97
:10044000EEC3E33CF17905E9F62733CCF29E118146
:100450007E80108A829F480DD7B4FC2FB5C7DD88F7
:10046000146B2B54EA1D945CB0EF1224CDEBE1E247
:1004700064733F0E5261253EF80F4BECC00030F61E
:1004800002493D106E20C9A62FFE2C2B752E452645
:10049000AB48A980FC04CCD3B5BAA338317D01D9CF
:1004A000A77B96B663694EF7DEE078CA50AA419101
:1004B0006588E42185DA3A27BE1C3E425E17527FEA
:1004C0001F89246F8F5C67740E12878DE934ED737A
:1004D000C4F8615B05DF594C97798318A45595EBF7
:1004E000BD53F5F15766469FB2810951862216DD4C
:1004F00023937629C2D71DD4BF363FEA4B1132B9B8
:10050000625460D66D439A0D929CB0EF586C9D7703
:100510002D70FAF3B30BE2407EF48AE58C3C567101
:10052000D164E1820ACB131590EC0399AF145D0FEF
:10053000334A94A5A8351BE36AC628FF4DE72584F6
:10054000AC08AEC5A22AB8370C7AA0C3CEAD061A45
:100550009E8BFBD5D0C11ED0B49BB144F247C76877
:10056000CF72BB4F5AF9DC6BDBD2E87CC8EE98A1A6
:10057000E6D839075FFD8E19B73BBCCD7CE38173AC
:10058000B211BF6F2098FE7596EF6CDA50E10972D8
:100590005445BA34805BED3E532C87A457F3333F68
:1005A0003CB767B4A325604F076B1B47150FE40AE0
:1005B000EAD1327836498D4BD2BCA5DC1D0D4DCD2C
:1005C0009A825FFC9465BEE2F4C91E44CB9E0C6423
:1005D000712663B314E840708A0E19426DAC88101E
:1005E0005CDF41A9ADE5FB74CCD5068E5986CE1FE4
:1005F0003D76E08FB977277BA6D829D3ECB813F7DF
:10060000FAC3516ADE4A5AEBC28B234892CF62A8E2
:1006100099F8D02E856143C8BDF00593CA4EF17D8F
:1006200030FDC469662F08B152F921E67A2BDD3915
:1006300084FFC091D637D47F2D9B5DA13B6EB5C59D
:100640004604F590EE7E831C0356B6AA00170135CA
:1006500055790B12BB1A31E7022816C1F6A2DB1836
:100660009C89683897ABC72AD73AF2C6244CB05851
:10067000A0225E9DD9A7E9AEAF8C959F28B720D761
:10068000B030C30919C067D6003C7EE7E9F4085AC8
:10069000F8B82E05A6259E5CD8150DE1F611546B11
:1006A000CD2146665E84AD06382944C5A2CEF1AAA6
:1006B000C1407186B5EFFC36A8CB0A48274564A334
:1006C000AF8CB2C69F0789DC17D34979FBFE1DD0DA
:1006D000B9884352BC01782B7D94C70EDEA5D59B0B
:1006E000CCF7617AC274813903AB96A037BD2D7205
:1006F000753FC9D48E6FF98DED62DB1CDF04AC1B36
:100700006C144B63D0BFB482EC7B1A5992D2106048
:10071000B63D5FE6806E70C4F235D97CEEE541A44B
:100720005B50DDBB4CF31F9D5D57555197E358421D
:100730004D9C73BAC877316926AEEA8ADA22B3874C
:1007400056FA930B341633E8E453BEA9B13A3EF59A
:10075000906ACF3B12FD8F9AA7479199EB0F24FF28
:100760002318854E7F0CE0A1D2D12C2A4A024F1EBD
:1007700095688B98836D76CA6532132FC3829AA4CD
:10078000BA8160373435FC80A8516567ED305F1061
:10079000D34A272F13B92AD2CCE1EFAEEBBEF4BD7A
:1007A000CF43B3C58884B7DD3940CE486D9B7261B5
:1007B0007EE7A14E532E773BE2C936221B6E73B102
:1007C00003B24C87A9D44D0FD8156CAA18F6495717
:1007D0005DFB7A149463A011B09EDE0546C8EE4717
:1007E000DBDC24899C919729E97BC1071EB8FDFEBB
:1007F000ACC662984FF179E0E86B7856B68D04503C
:1008000086CA6F20E6EAE576171C747FBC0D2C853E
:10081000F76696E48B753F4BD938AF7CDA0B832DA6
:100820003132A2F51D594145BF3C1FF8F98AD01657
:10083000256912999D2195AB01A6D7B5C07DFF58BA
:100840000E3A92D155E3089FD63E528EFAA3C702C4
:10085000CDDF8F64198CF3A70C5E0A6A09F0935BF5
:1008600042C20623EC71ADB4CBBB7028D51A5C3301
:10087000685A004490A5C4263D2BF25496ADDA1F69
:10088000ED33E18169080D0ADB35779A64D1FC7894
:10089000AA1BD067A0DDFA6C63710584176A894FC3
:1008A000667FC65055926FBDE7D240728DBBEC0695
:1008B000428AE4889D7E7A822713411AAFC8A476C3
:1008C000B4C2FE6D1CD96130B37CEAF7290FF23B4C
:1008D00051C1DE5FE52A2F990B5DA32B4AAB95A58D
:1008E000D35856EE283100CC1546CAE686383C650A
:1008F000F5E39FD65B094983702D53A97DE2C4AC13
:100900008E5EB825F4B957F3F16847B2A25920CEEC
:1009100034795C900E1EBED52223B1C91862162E02
:10092000913E078FD83F933DD49BDF8521FB117407
:1009300097C7D7DC4C194598E943024BBCC3049CCC
:100940006BF07552A726F6C5BACFB0B7AE5AA1BFA5
:10095000038B80126E0CEBF9C04424EF10F8A88CC6
:10096000E87BFF9E2CCD603687B594A654733A146D
:100970004E011DB6FD37484D39CBE0320000000076
:100980000000000000000000000000000000000067
:100990000000000000000000000000000000000057
:1009A0000000000000000000000000000000000047
:1009B0000000000000000000000000000000000037
:1009C0000000000000000000000000000000000027
:1009D0000000000000000000000000000000000017
:1009E0000000000000000000000000000000000007
:1009F00000000000000000000000000000000000F7
:100A000000000000000000000000000000000000E6
:100A100000000000000000000000000000000000D6
:100A200000000000000000000000000000000000C6
:100A300000000000000000000000000000000000B6
:100A400000000000000000000000000000000000A6
:100A50000000000000000000000000000000000096
:100A60000000000000000000000000000000000086
:100A7000000000000000000000000000A877A6E0D1
:100A8000F7435A3585E272978FB71A6287380D6738
:100A9000C7BE4F3E2076378F68B7A9263F2B10E39D
:100AA000307E900E850A11241FBECFEFD4E0DEBF4A
:100AB000CDBF11E0A0E0B1E0E0EDF5E302C00590AC
:100AC0000D92AA3EB107D9F724E0AAEEB1E001C029
:100AD0001D92A43AB207E1F70E94CD180C94E61AD1
:100AE0000C94000081E08093EC010895E82FF0E081
:100AF000E050FE4F80810895882311F085EC01C0FD
:100B000085E88093BC000895262F30E0982F01C01F
:100B100096956A95EAF73195219531092770332723
:100B200001C0880F2A95EAF7892B08958F929F922A
:100B3000BF92CF92DF92EF92FF920F931F93CF93CA
:100B4000DF93CDB7DEB766970FB6F894DEBF0FBE62
:100B5000CDBFE12CF12C00E010E0DE01519680E0E9
:100B600090E0F701E80FF91FE458F54FE491ED9399
:100B7000019686309105A9F7DE01119680E090E09C
:100B8000FC01EA5EFC4FE081F0E0E458FF4FE491A5
:100B9000ED9301968A30910599F7EB814E813A8564
:100BA0005D81898984279E2F9770692F70E0B82E08
:100BB00001C0B6949A95EAF77195619571096770CD
:100BC000772701C0880F6A95EAF78B29831B852751
:100BD0008B8729819A81F8858A898927A22FA77016
:100BE0006A2F70E0B82F01C0B695AA95EAF7719503
:100BF000619571096770772701C0880F6A95EAF7D8
:100C00008B2B841B8F278C87BF81A985A7706A2FA8
:100C100070E08B89C82ECB26DC2C0A2E01C0D6941E
:100C20000A94EAF77195619571094B0187E0882272
:100C300099248C2D082C01C0880F0A94EAF78D297D
:100C40008E1B82278D878C812C8925277F2F77709B
:100C5000C72ED12C622F01C066957A95EAF7D19400
:100C6000C194D10877E0C722DD2401C0220FCA94C5
:100C7000EAF7262B281B2E272E872D899227B7705F
:100C8000CB2ED12C292F01C02695BA95EAF7D19405
:100C9000C194D108B7E0CB22DD2401C0990FCA94DA
:100CA000EAF7922B981B95279F879E898F2F89277C
:100CB000982F01C09695AA95EAF701C0880F8A94EB
:100CC000EAF7892B841B8327888B46E050E060E19C
:100CD00073E0CE010B960E94971A98012F5F3F4F49
:100CE000892B59F0890126E0E20EF11C073011052D
:100CF00009F033CF1092200339C180911403322FB1
:100D00002227F901E80FF11DE458FF4F4491C80173
:100D1000029650911903982F8827FC01E50FF11DC9
:100D2000E458FF4FE491E427E09308034091120355
:100D3000F901E40FF11DE458FF4F449150911B035A
:100D4000FC01E50FF11DE458FF4FE491E427E09327
:100D5000090340911503F901E40FF11DE458FF4F19
:100D6000449150911D03FC01E50FF11DE458FF4F24
:100D7000E491E427E0930A0340911003F901E40FA2
:100D8000F11DE458FF4F449150911803FC01E50F09
:100D9000F11DE458FF4FE491E427E0930B034091E9
:100DA0001103F901E40FF11DE458FF4F44915091F4
:100DB0001A03FC01E50FF11DE458FF4FE491E4270D
:100DC000E0930C0340911303F901E40FF11DE45883
:100DD000FF4F449150911F03FC01E50FF11DE458B2
:100DE000FF4FE491E427E0930D0340911603F901CE
:100DF000E40FF11DE458FF4F449150911C03FC0196
:100E0000E50FF11DE458FF4FE491E427E0930E0352
:100E100040911703F901E40FF11DE458FF4F44918D
:100E200050911E03FC01E50FF11DE458FF4FE491C2
:100E3000E427E0930F0340911003F901E40FF11D43
:100E4000E458FF4F449150911703FC01E50FF11D49
:100E5000E458FF4FE491E427E09300034091150329
:100E6000F901E40FF11DE458FF4F449150911A032A
:100E7000FC01E50FF11DE458FF4FE491E427E093F6
:100E8000010340911303F901E40FF11DE458FF4FF2
:100E9000449150911603FC01E50FF11DE458FF4FFA
:100EA000E491E427E093020340911203F901E40F77
:100EB000F11DE458FF4F449150911F03FC01E50FD1
:100EC000F11DE458FF4FE491E427E09303034091C0
:100ED0001403F901E40FF11DE458FF4F44915091C0
:100EE0001D03FC01E50FF11DE458FF4FE491E427D9
:100EF000E093040340911103F901E40FF11DE4585C
:100F0000FF4F449150911E03FC01E50FF11DE45881
:100F1000FF4FE491E427E093050340911903F901A1
:100F2000E40FF11DE458FF4F449150911B03FC0165
:100F3000E50FF11DE458FF4FE491E427E093060329
:100F400040911803F901E40FF11DE458FF4F24917B
:100F500030911C03830F911DFC01E458FF4FE49175
:100F6000E227E093070381E08093200366960FB6A3
:100F7000F894DEBF0FBECDBFDF91CF911F910F91CF
:100F8000FF90EF90DF90CF90BF909F908F9008954B
:100F9000863028F4E0912103F0912203099408950A
:100FA00090EC980F963098F480E490E049E450E09B
:100FB000FA01E81BF90BDC01A050BE4F2C91EA5E50
:100FC000FC4F208301968634910591F708959AEBA2
:100FD000980F9630C8F4809146028093190380914F
:100FE00047028093180380914802809317038091F1
:100FF00049028093160380914A02809315038091E1
:101000004B0280931403089594EB980F9430C0F42E
:1010100090914C029093130390914D029093120380
:1010200090914E029093110390914F029093100370
:1010300070E0680F711D6035710511F40C94960510
:101040000895462F50E0BC0180E092E00C94A41A71
:10105000EF92FF920F931F93CF93DF937C01CB010D
:10106000D22FC32F1093220300932103642F0E94D9
:1010700021081092F00286E0F701AEEEB1E0019097
:101080000D928A95E1F786E0EEEEF1E0AAEFB2E08C
:1010900001900D928A95E1F7ED2FFC2F80E290E010
:1010A0002191DC01A050BE4F2C9301968034910514
:1010B000B9F7459844981092FF011092FE0184EA16
:1010C0008093BA0081E48093BC00DF91CF911F919F
:1010D0000F91FF90EF9008958091ED010895809118
:1010E000ED01811108C08091BC0084608093BC0038
:1010F00081E08093ED0108958091FA010895FC014B
:1011000096E0A4EFB1E001900D929A95E1F781E0AD
:101110008093FB0108951F920F920FB60F92112436
:101120002F933F934F935F936F937F938F939F93EF
:10113000AF93BF93EF93FF938091B900887F80397D
:1011400051F188F4803721F128F4803609F188368E
:10115000F9F0D2C08038F9F0883809F4CDC088376A
:1011600009F0CAC015C0803B09F48BC038F4803A3E
:1011700009F47BC0883A09F0BFC083C0803C09F401
:10118000B9C0883C09F4B6C0883B09F482C0B4C039
:101190001092FD01AFC08091FD01882309F458C071
:1011A0008091BB002091FE013091FF01203F31056D
:1011B00089F4853511F08A3A69F41092200396E09B
:1011C000EEEEF1E0AAEFB2E001900D929A95E1F710
:1011D0001092FA012091FE013091FF01232B91F42E
:1011E000843681F49091FB01992361F096E0E4EF5D
:1011F000F1E0AAEFB2E001900D929A95E1F791E04B
:101200009093FA01909120039923D1F02091FE014F
:101210003091FF01E091FE01F091FF01E770FF279F
:10122000E050FD4F4081E091FE01F091FF01E77039
:10123000FF27E85FFC4F90818427890FF90104C0E4
:10124000E091FE01F091FF01E050FE4F808344C029
:101250008091BB0090E09093FF018093FE0181E0BC
:101260008093FD011092FC0145C06091FC018091CA
:10127000FE019091FF019091FC01891B0E94D00713
:1012800039C08091FE019091FF010E94C807109221
:10129000FC0180912003E091FE01F091FF01E050FC
:1012A000FE4F8823B1F08081E091FE01F091FF01B3
:1012B000E770FF27E85FFC4F2081E091FE01F0918D
:1012C000FF01E770FF27E050FD4F9081821B8927C7
:1012D00001C080818093BB008091FE019091FF014D
:1012E00001969093FF018093FE018091FC018F5F36
:1012F0008093FC0185EC01C085E88093BC00FF91E0
:10130000EF91BF91AF919F918F917F916F915F917D
:101310004F913F912F910F900FBE0F901F901895F6
:10132000FC01892B01F18091260390912703292F3D
:101330002F702F3021F421E02093230302C010925C
:10134000230320912303222329F093E090838183B8
:10135000828309C022E02083282F30E0392B32839A
:101360002183838394838091260390912703909314
:10137000250380932403089542E050E064E273E083
:1013800086E293E00E94971A0895419A80E38A9535
:10139000F1F7419828E030E080E098E19A95F1F784
:1013A0004098880F329B816098E19A95F1F7409AB6
:1013B0002150310991F78093260328E030E098E12D
:1013C0009A95F1F74098880F329B816098E19A9541
:1013D000F1F7409A2150310991F78093270380E07B
:1013E0000895CF93CFB7F894399A389A3A98429A99
:1013F000409A41980E94C509CFBF80E0CF910895DF
:101400008EE391E008958823C1F091E0E82F880FE2
:10141000FF0B292F30E0241735076CF4DB01A20FF6
:10142000B31F2C9130E0E217F3071CF48FEF890F04
:1014300008959F5FEECF8FE1089580E0089540E228
:1014400050E0623041F0633019F06AE871E005C0A5
:101450006AE671E002C06AE471E00C94030ADC0100
:10146000892B39F093E1EBE3F3E001900D929A952B
:10147000E1F783E1EBE3F3E0A8E2B3E001900D9242
:101480008A95E1F708959C019091B601953069F035
:10149000992359F0232B21F0933039F082E003C0D7
:1014A000913019F084E08093B60108951F93CF9393
:1014B000DF931F92CDB7DEB785E08093B6011FE0C2
:1014C0002FE389E191E0215080409040E1F700C096
:1014D0000000198261E070E0CE0101960E94B20B1B
:1014E000489721F0115061F780E001C081E00F9032
:1014F000DF91CF911F91089543E150E068E273E0DE
:101500008BE393E00E94971A08951F93CF93DF9384
:10151000CDB7DEB7A6970FB6F894DEBF0FBECDBF2E
:10152000198261E070E0CE0101960E94B20B883111
:1015300019F01092B601FFC08091B703882331F0F3
:101540008091B601853011F41092B6018091B703F5
:10155000811103C085E08093B6018091B60182308D
:10156000E1F0843099F1811149C083E0898380E8FA
:101570008A8381E08B8342E250E060E870E0CE0134
:1015800004960E94AD1A63E270E0CE0101960E94BB
:10159000B20B882399F184E02FC013E0198380EC0B
:1015A0008A838BE18B8340E250E061E070E0CE0102
:1015B00004960E94AD1A63E270E0CE0101960E948B
:1015C000B20B8823D9F01093B60118C083E0898349
:1015D00080EC8A838BE18B83FE01349680E2DF010D
:1015E0001D928A95E9F763E270E0CE0101960E94B0
:1015F000B20B882319F081E08093B60181E08983E2
:1016000061E070E0CE0101960E94B20B803209F0D9
:1016100092C084E080933B0320E030E080E090E0E3
:1016200041E050E0FC01E056FC4F6081662349F048
:10163000BA01082E02C0660F771F0A94E2F7262B24
:10164000372B01968031910569F730933F03209342
:101650003E0390E020E030E060E870E0F901E05502
:10166000FC4F8081882341F0AB01022E02C05595CA
:1016700047950A94E2F702C040E050E0942B2F5FB8
:101680003F4F2830310551F7998380E020E030E06A
:1016900060E870E0F901E854FC4F4081442341F0D8
:1016A000AB01022E02C0559547950A94E2F702C09D
:1016B00040E050E0842B2F5F3F4F2830310551F739
:1016C0008A8390933C0380933D03903819F491E80A
:1016D00090933C03803819F481E880933D0384E0C3
:1016E000E0E4F3E0DF011D928A95E9F780E090E005
:1016F00040E850E0FC01E056FC4F20812223A9F095
:10170000FC0123E0F595E7952A95E1F7E55CFC4FB0
:101710009C0127703327BA0102C0759567952A95F9
:10172000E2F79B013581232B2583019680329105B9
:1017300009F780E001C08FEFA6960FB6F894DEBFE0
:101740000FBECDBFDF91CF911F9108950E94850AF2
:1017500080E008958AEA91E008953B984398249A9E
:101760002C9808950F931F93662309F44BC0FC0136
:10177000860F911DBC0180E090E09C01E617F70701
:1017800081F0089640E850815423D901A056BC4FFF
:101790005C932F5F3F4F469582179307A1F73196D1
:1017A000ECCFE0EAF3E0CF93DF93EF93FF93019167
:1017B000002311F049F416C000003B9A19E00FD045
:1017C0003B980197A1F70EC03B9A11E008D03B98D7
:1017D00015E005D000000000019749F703C01A95F5
:1017E000F1F708950000FF91EF913B9ADF91CF91BF
:1017F00000000000000000003B980FEF0A9511F078
:10180000339BFCCFE0EAF3E0EF93FF93332700270D
:101810000395A1F03399FCCF08C004E6039572F05C
:101820003399FCCF339551F0019304E6039532F0E0
:10183000339BFCCF339511F00193EFCFFF91EF91E4
:10184000832F90E00097B1F030FF14C020E0DF015B
:101850006081518141E0651708F040E04D93329678
:101860002F5F3213F5CF24E12A95F1F70197959573
:10187000879502C080E090E01F910F910895CF936B
:10188000DF931F92CDB7DEB7198261E070E0CE0121
:1018900001960E94B20B009709F1489711F58091CB
:1018A000A403882311F088E001C080E09091A50393
:1018B000911184609091A603911182609091A70389
:1018C000911181608A3028F4883028F4853061F0E5
:1018D00008C08B3031F482E090E008C080E090E0F6
:1018E00005C083E090E002C081E090E00F90DF91BE
:1018F000CF910895DC01892B39F093E1E6E6F3E01E
:1019000001900D929A95E1F7089543E150E063E567
:1019100073E086E693E00E94971A0895CF93DF93D1
:1019200085E08093660320E030E080E090E041E0D5
:1019300050E0FC01E056FC4F6081662349F0BA019B
:10194000082E02C0660F771F0A94E2F7262B372B6A
:1019500001968031910569F730936E0320936D03F2
:10196000E0E080E090E040E850E0DC01A055BC4FB2
:101970002C91222341F09A01082E02C0359527951B
:101980000A94E2F702C020E030E0E22B01968830B2
:10199000910559F720E080E090E060E870E0DC011C
:1019A000A854BC4F3C91332341F0AB01082E02C038
:1019B000559547950A94E2F702C040E050E0242B89
:1019C00001968830910559F780E040E050E0A0E8AA
:1019D000B0E0EA01C054DC4F9881992341F0BD0189
:1019E000042E02C0759567950A94E2F702C060E084
:1019F00070E0862B4F5F5F4F4830510551F7809361
:101A0000690390E040E050E0A0E8B0E0EA01C8538C
:101A1000DC4F3881332341F0BD01042E02C075959F
:101A200067950A94E2F702C060E070E0962B4F5F82
:101A30005F4F4830510551F7309152033323A9F0DD
:101A400030915103E31BE093670330915003231B54
:101A50002093680320914F03821B80936903809138
:101A60004E03981B90936A0313C0E0935103209395
:101A7000500380934F0390934E031092670310928C
:101A800068031092690310926A0381E08093520305
:101A900080E090E030E060E870E0FC01E053FC4F53
:101AA0002081222341F0AB01082E02C055954795B5
:101AB0000A94E2F702C040E050E0342B01968830EF
:101AC000910559F730936B0380E090E020E060E8E7
:101AD00070E0FC01E852FC4F4081442341F0AB012F
:101AE000082E02C0559547950A94E2F702C040E0DF
:101AF00050E0242B01968830910559F720936C0310
:101B00008091D2018823B1F0333348F080916D0386
:101B100090916E03926090936E0380936D032333D4
:101B200048F080916D0390916E03946090936E03E2
:101B300080936D0388E0EFE6F3E0DF011D928A9564
:101B4000E9F780E090E040E850E0FC01E056FC4F0F
:101B500020812223A9F0FC0123E0F595E7952A9541
:101B6000E1F7EA59FC4F9C0127703327BA0102C004
:101B7000759567952A95E2F79B013185232B21877F
:101B800001968034910509F7DF91CF910895CF93A5
:101B9000DF93CDB7DEB728970FB6F894DEBF0FBE40
:101BA000CDBF80E4898383E08A831B8263E070E099
:101BB000CE0101960E94B20B803421F40E948E0C5B
:101BC00080E001C081E028960FB6F894DEBF0FBE1A
:101BD000CDBFDF91CF910895109252030E94C70D9F
:101BE00091E0811190E0892F08950E94C70D80E057
:101BF000089587EB91E00895F999FECF40E150E018
:101C000060E070E08AE793E00E94C41AF999FECF81
:101C1000089580E1E3ECF1E0AAE7B3E001900D92D2
:101C20008A95E1F70C94FC0DF999FECF40E150E064
:101C300060E070E08AE793E00E94B41AF999FECF61
:101C400049E050E060EE71E08AE793E00E94971A65
:101C5000892BA1F080E1EAE7F3E0DF011D928A958C
:101C6000E9F789E0E0EEF1E0AAE7B3E001900D9238
:101C70008A95E1F70E94FC0D0C94090E80E1EAE7D9
:101C8000F3E0A3ECB1E001900D928A95E1F708959D
:101C900020917903211104C0FC0160830C94090E8A
:101CA0000895FF920F931F93CF93DF93EC018B0165
:101CB00081E1FB0111928A95E9F741305105B1F4B8
:101CC0008091CC01883059F06091CD0170E089811C
:101CD0000E94F516F82E6091CD0170E012C0898146
:101CE00040E2F42EF80E8A81805E24C04230510515
:101CF00061F462E070E089810E94F516F82E62E0DE
:101D000070E08A810E94F51615C08981082E000CAA
:101D1000990B80589F4F9595879595958795F82EA7
:101D20008A81082E000C990B80589F4F95958795B6
:101D3000959587954C81042E000C550B40585F4FAC
:101D400093E0559547959A95E1F79D8195959595E1
:101D500095955E812B81022E000C330B20583F4F4E
:101D600063E0359527956A95E1F7B901E3E0660FE1
:101D7000771FEA95E1F7607CF62AF801F082B90155
:101D8000A5E0660F771FAA95E1F7607C862B81831B
:101D9000692F6871F4E06F9FB00111243695322FDE
:101DA000222737952795262B242BF8012283F0E252
:101DB0009F9FC0011124952F969596959695892BF6
:101DC000F80183838885809584838F8180958583BE
:101DD00082E5868389859A8590878783D8011996BD
:101DE000FE013B9688E001900D928A95E1F7DF9124
:101DF000CF911F910F91FF9008950F931F93CF9351
:101E0000DF93EC01FB0181E1DB011D928A95E9F78B
:101E100039812A814130510521F48091CD018130F1
:101E200021F4305880E8820F14C040E83403C00128
:101E300011240FE510E0B8010E94691A30E8360F4E
:101E400040E82403C0011124B8010E94691A80E807
:101E5000860F2B8120589C8190585D814E81308364
:101E6000218382839383148255834683888580955A
:101E700087838F8180958087DF91CF911F910F910C
:101E800008950F931F93CF93DF93EC01FB0181E142
:101E9000DB011D928A95E9F739812A81413051058C
:101EA00021F48091CD01813021F4305880E8820FF7
:101EB00014C040E83403C00111240FE510E0B8015C
:101EC0000E94691A30E8360F40E82403C00111244B
:101ED000B8010E94691A80E8860F2B8120589C81E6
:101EE00090585D814E813083218382839383548314
:101EF00045838885809586838F8180958783DF9150
:101F0000CF911F910F9108952130310529F0223092
:101F1000310521F00C94510E0C94FD0E0C94410FE0
:101F2000EF92FF920F931F93CF93DF938C01EB01FE
:101F30008091D101882321F094E8E92EF12C03C08F
:101F400084E0E82EF12C83E1FE0111928A95E9F7F5
:101F5000F8018081843009F47CC330F4823069F068
:101F6000833009F4F5C03AC7863009F41FC508F478
:101F700042C1873009F4E5C431C783E5898786E427
:101F80008A87F801838194819C878B879091CF0108
:101F90008181992379F086FF05C08F8198858064BF
:101FA00098878F83F801818187FF28C08F8198856A
:101FB000806122C087FF05C08F81988580649887E3
:101FC0008F83F801818186FF05C08F8198858062AB
:101FD00098878F83F8018181928197FF05C08F8157
:101FE0009885806198878F83F8018181928196FF1F
:101FF00005C08F819885886098878F839091D001E4
:10200000F80181819923B9F083FF02C084E68A83B5
:10201000F801818182FF02C08CE98A83F801818105
:1020200081FF02C08CE98983F801818180FF25C08E
:1020300084E6898322C083FF05C08F8198858160F3
:1020400098878F83F801818182FF05C08F819885F1
:10205000906498878F83F801818181FF05C08F810B
:102060009885826098878F83F801818180FF05C001
:102070008F819885906898878F83F801818185FF8B
:1020800005C08F819885906198878F83F801818141
:1020900084FF05C08F819885946098878F83F801AD
:1020A0008181928195FF05C08F8198859062988784
:1020B0008F83F8018181928194FF05C08F8198857B
:1020C000926098878F83F8018181928188739073E1
:1020D0008833904331F41092CF011092D0010E94C6
:1020E000090EF80181819281847390738433904347
:1020F00039F481E08093CF011092D0010E94090E43
:10210000F80181819281827390738233904339F414
:1021100081E08093D0011092CF010E94090EF80156
:1021200081819281807199270E943517882329F037
:102130008F819885986098878F838F81988595FF88
:1021400002C02FEF2D8391FF49C68FEF8E8346C6C5
:1021500086E4898783E48A87F80182818B8781817D
:1021600087FF05C08F819885806198878F83F801EC
:10217000818186FF05C08F819885806498878F83D1
:10218000F801818185FF05C08F81988590619887CE
:102190008F83F801818184FF05C08F8198859460C9
:1021A00098878F83F801818183FF05C08F8198858F
:1021B000816098878F83F801818182FF05C08F81BC
:1021C0009885906498878F83F801818181FF05C08D
:1021D0008F819885826098878F83F801818180FF45
:1021E00005C08F819885906898878F83F8018181D9
:1021F000807190E050C487E4898783E48A8788E00F
:10220000F8013996DE011B9601900D928A95E1F74F
:10221000F8018781442329F083FF03C091E0909364
:1022200079039091CE01923009F47CC028F499236F
:1022300061F09130C1F170C1943009F4EEC008F43E
:10224000ADC0953009F428C167C187FF05C08F81F3
:102250009885806198878F83F801878186FF05C004
:102260008F819885806498878F83F801878185FFA7
:1022700005C08F819885886098878F83F801878152
:1022800084FF05C08F819885806298878F83F801CD
:102290008781908593FF33C08F819885E82AF92A3A
:1022A000F886EF822CC086FF05C08F8198858062FA
:1022B00098878F83F801878187FF05C08F81988574
:1022C000806498878F83F801878184FF05C08F81A0
:1022D0009885886098878F83F801878185FF05C07E
:1022E0008F819885806198878F83F8018781908599
:1022F00093FF05C08F819885906198878F83F8013F
:102300008781908591FF05C08F819885906298871D
:102310008F83F8018781908592FFFEC08F81988519
:102320009260F8C087FF05C08F819885806198878B
:102330008F83F801878186FF05C08F81988580642F
:1023400098878F83F801878185FF05C08F819885E5
:10235000886098878F83F801878184FF05C08F810B
:102360009885806298878F83F8018781908593FF95
:1023700005C08F819885926098878F83F801878147
:10238000908591FF05C08F819885806898878F839D
:10239000F8018781908592FFBFC07AC087FF05C092
:1023A0008F819885846098878F83F801878186FF65
:1023B00005C08F819885806198878F83F801878118
:1023C00085FF05C08F819885806498878F83F80189
:1023D000878184FF05C08F819885886098878F8367
:1023E000F8018781908593FF05C08F81988580646F
:1023F00098878F83F8018781908591FF05C08F8131
:102400009885806898878F83F8018781908592FFEF
:1024100083C08F81988580627DC087FF05C08F81D2
:102420009885806498878F83F801878186FF05C02F
:102430008F819885806298878F83F801878185FFD7
:1024400005C08F819885806198878F83F801878187
:1024500084FF05C08F819885886098878F83F801F5
:102460008781908591FF05C08F81988590629887BC
:102470008F83F8018781908592FF05C08F819885B1
:10248000926098878F83F8018781908593FF44C07D
:102490008F81988584603EC087FF05C08F819885B5
:1024A000806198878F83F801878186FF05C08F81BF
:1024B0009885886098878F83F801878185FF05C09C
:1024C0008F819885926098878F83F801878184FF38
:1024D00005C08F819885806498878F83F8018781F4
:1024E000908591FF05C08F819885806898878F833C
:1024F000F8018781908592FF05C08F81988584605F
:1025000098878F83F8018781908593FF05C08F811D
:102510009885906198878F83F801878183FF05C034
:102520008F819885946098878F83F8018781908543
:1025300094FF05C08F819885816098878F83F8010B
:102540008781908595FF05C08F81988590649887D5
:102550008F83F8018781908597FF05C08F819885CB
:10256000826098878F83F8018781908596FF05C0E8
:102570008F819885906898878F83F80181818983FE
:1025800082818A8383818B8384818C8385818D83FF
:1025900086818E83878190859C01207F3071203FCA
:1025A000304111F460E007C09C01207F3072203F71
:1025B000304231F461E08EEC91E00E94480E43C05D
:1025C0009C01207F3078203F304811F462E0F3CF47
:1025D0009C01207F3074203F304411F463E0EBCF46
:1025E0009C01207F3870203F384079F4F8018381C6
:1025F000803C2CF464E08EEC91E00E94480EF801DF
:102600008381813404F165E0D6CF9C01207F327054
:10261000203F324089F480918D03811114C081E004
:102620009091D201911180E08093D2010E94090E15
:1026300081E080938D0307C0807F9927803F9105BB
:1026400011F010928D03F801878190858870992789
:1026500022C286E3898784E38A8784E0F80135967D
:10266000DE011B9601900D928A95E1F7F8018381B6
:102670009481442329F083FF03C021E02093790350
:102680009C0124713C7024313C4011F460E042C054
:102690009C0124723C7024323C4011F461E03AC049
:1026A0009C0124743C7024343C4011F462E032C03C
:1026B0009C0124783C7024383C4011F463E02AC02B
:1026C0009C0124703C7124303C4111F464E022C030
:1026D0009C0124703C7224303C4211F465E01AC025
:1026E0009C0124703C7424303C4411F466E012C018
:1026F0009C0124703C7824303C4811F467E00AC007
:1027000084709C7084309C4049F4F80182818E3C36
:102710002CF469E08CEC91E00E94480E80917903E2
:10272000811134C0F801838194819C0125703C7033
:1027300025303C4011F483E006C086709C708630E2
:102740009C4029F481E08093CD010E94090EF8019C
:102750008381948184709C7084309C40A9F4F8013A
:10276000828183339CF080918D0381110FC081E0C1
:102770009091D101911180E08093D1010E94090EC6
:1027800081E080938D0302C010928D03F801838154
:1027900080FF05C08F819885806198878F83F801BD
:1027A000838181FF05C08F819885806498878F839E
:1027B000F801838183FF05C08F8198859460988795
:1027C0008F838091CC01883029F1F801938194FFA7
:1027D00005C02F813885216038872F83F8019381C8
:1027E00095FF05C02F813885306438872F83F80125
:1027F000938196FF05C02F813885226038872F830B
:10280000F801938197FFACC12F81388530683887F4
:102810002F83A6C1F801938192FF06C02F813885CE
:10282000E22AF32AF886EF82F8012381348133FF0C
:1028300005C02F813885326038872F83F8012381C6
:10284000348132FF05C02F813885306238872F836D
:10285000F801238134812474307F2434304F29F4EB
:102860002F813885286238872F83883031F1863070
:1028700009F44EC1893009F44BC1843009F448C1D0
:10288000F8018381948194FF02C084E68C83F8016F
:102890008381948195FF02C08CE98C83F801838148
:1028A000948196FF02C08CE98B83F8018381948127
:1028B00097FF2EC184E68B832BC1F80123813481DD
:1028C00080918C0334FF09C080FD0AC090918B0376
:1028D0009F5F90938B03816001C08E7F80938C03F8
:1028E00080918C0335FF09C081FD0AC090918B0354
:1028F000915090938B03826001C08D7F80938C03F5
:1029000080918C0336FF09C082FD0AC090918A0332
:102910009F5F90938A03846001C08B7F80938C03B8
:1029200080918C0337FF09C083FDFDC090918A031D
:10293000915090938A03886001C0877F80938C03B5
:10294000F2C0F801818180FF05C08F819885816088
:1029500098878F83F801818181FF05C08F819885D9
:10296000906498878F83F801818182FF05C08F81F1
:102970009885826098878F83F801818183FF05C0E5
:102980008F819885906898878F83F801818184FF73
:1029900005C08F819885806498878F83F801818135
:1029A00085FF1CC28F81988580617DC0F80181817F
:1029B00080FF05C08F819885816098878F83F8019B
:1029C000818181FF05C08F819885906498878F836E
:1029D000F801818182FF05C08F8198858260988788
:1029E0008F83F801818183FF05C08F81988590686E
:1029F00098878F83F801818186FF05C08F81988534
:102A0000806298878F83F801818184FF05C08F8160
:102A10009885806498878F83F801818185FF05C040
:102A20008F819885806198878F83F801818187FFE6
:102A300005C08F819885906298878F83F801818186
:102A4000928190FF05C08F819885886098878F83D9
:102A5000F8018181928191FF05C08F8198859260F4
:102A600098878F83F8018181928192FF05C08F81C1
:102A70009885946098878F83F8018181928193FF74
:102A800005C08F819885846098878F83F801818144
:102A90009281882794700E943517882309F49EC17B
:102AA0008F819885986098878F8398C1F80183817A
:102AB000948192FF06C08F819885E82AF92AF886CA
:102AC000EF82F8018381948193FF05C08F819885FF
:102AD000926098878F83F801838182FF05C08F8180
:102AE0009885906298878F83F8018381948196FFFF
:102AF00005C08F819885806298878F83F8018381D4
:102B0000948197FF05C08F819885886098878F830F
:102B1000F8018181898382818A83F801838194818C
:102B20008870992701CB24FF03C080918B038A838F
:102B3000F801838185FF04C080918B0381958A838E
:102B4000F801838186FF03C080918A038983F8019D
:102B5000838187FFE2CF80918A0381958983DDCFCE
:102B6000482F50E04A30510508F081CEFA01EC5C64
:102B7000FF4F0C947D1AF801838182FF05C08F817D
:102B80009885906298878F83F8018381948193FF61
:102B900005C08F819885926098878F83F801838123
:102BA000948192FF6DCE8F819885E82AF92AF88664
:102BB000EF8266CEF801838182FF05C08F81988500
:102BC000906298878F83F8018381948193FF05C079
:102BD0008F819885926098878F83F8018381948193
:102BE00092FF4ECE8F8198859064A6C0F8018381B4
:102BF000948192FF05C08F819885906498878F8318
:102C0000F8018381948193FF06C08F819885E82A1B
:102C1000F92AF886EF82F801838182FF05C08F814F
:102C20009885926298878F83F8018381948196FFBB
:102C300005C08F819885806298878F83F801838192
:102C4000948195FF1DCE8F819885886075C0F801AD
:102C50008381948192FF05C08F81988590629887C7
:102C60008F83F8018381948193FF05C08F819885BC
:102C7000926098878F83F801838182FF01CE8F81D4
:102C80009885906259C0F8018381948192FF05C0B4
:102C90008F819885906898878F83F80183819481CC
:102CA00093FF05C08F819885926098878F83F80184
:102CB000838182FF05C08F819885906298878F837A
:102CC000F8018381948195FF05C08F819885886084
:102CD00098878F83F8018381948196FF05C08F8147
:102CE0009885806298878F83F8018381948197FF0C
:102CF0000FCF8F819885E82AF92AF886EF8208CFCE
:102D0000F8018381948192FF06C08F819885E82A1B
:102D1000F92AF886EF82F8018381948193FF05C038
:102D20008F819885926098878F83F801838182FFD5
:102D3000A7CD8F819885886298878F83A1CDF80170
:102D4000838182FF06C08F819885E82AF92AF88658
:102D5000EF82F8018381948193FF05C08F8198856C
:102D6000926098878F83F8018381948192FF05C0D8
:102D70008F819885906298878F838F8198858F7ACD
:102D800098878F83F801238120FF03C08064988790
:102D90008F83F801838181FF05C08F8198858062D0
:102DA00098878F83F8018381948196FF05C08F8176
:102DB0009885886098878F83F8018381948195FF37
:102DC00005C08F819885806198878F83F801838102
:102DD000948194FF6ACD84E68C8367CDDF91CF9197
:102DE0001F910F91FF90EF90089587FD04C00E94FE
:102DF0001F0A805E089581950E941F0A90E2981B29
:102E0000892F08959C0180919503882311F08150AA
:102E100023C0909194039F5F9093940395312CF07D
:102E200010929303109294031BC040919103509110
:102E300092032417350739F0909193039F5F909385
:102E40009303109294039091930396304CF0109258
:102E500093031092940384E18093950381E0089595
:102E6000309392032093910308959C0180918F03E6
:102E7000909190038217930759F090918E039F5F72
:102E800090938E03953030F03093900320938F030E
:102E900010928E0380918F03909190030C940217EF
:102EA00026B183B1237090E1299F900111248F7086
:102EB000822B0895DC01892B81F095E0EBE9F3E0AA
:102EC00001900D929A95E1F785E0EBE9F3E0A6E930
:102ED000B3E001900D928A95E1F7089545E050E046
:102EE00066E973E08BE993E00E94971A0895EF92E8
:102EF000FF920F931F93CF93DF93EC01429A80E5EB
:102F00008A95F1F70E945017182F8091DF018230C7
:102F100028F418838FEF89838A832DC0429890E527
:102F20009A95F1F70E945017E82E429A80E58A950B
:102F3000F1F7429890E59A95F1F70E945017F82E14
:102F4000429A80E58A95F1F7429890E59A95F1F7D3
:102F50000E945017082F429A80E58A95F1F70E9447
:102F60005017429890E59A95F1F7429A1883E982B2
:102F70008A83FB820C83DF91CF911F910F91FF9089
:102F8000EF900895CF93DF9300D000D01F92CDB77C
:102F9000DEB7CE0101960E947717898180952A813C
:102FA00020959B81909535E0EBE9F3E0DF011D92E0
:102FB0003A95E9F780FF06C041E050E050939D0349
:102FC00040939C0381FF09C040919C0350919D0355
:102FD000426050939D0340939C0382FF09C040913F
:102FE0009C0350919D03446050939D0340939C0328
:102FF00083FF09C040919C0350919D03486050930A
:103000009D0340939C036091DF01382F30718072E3
:10301000623008F45BC046E040939B0324FF09C084
:1030200040919C0350919D03406450939D034093B5
:103030009C03332349F040919C0350919D034061D0
:1030400050939D0340939C03882349F040919C0337
:1030500050919D03406250939D0340939C0325FF34
:1030600009C020919C0330919D03346030939D03EF
:1030700020939C03633009F042C092FF09C0209165
:103080009C0330919D03206830939D0320939C0303
:1030900091FF09C020919C0330919D0331603093D2
:1030A0009D0320939C0390FF09C020919C033091C5
:1030B0009D03326030939D0320939C0393FF1FC0B8
:1030C00080919C0390919D03986015C097E0909328
:1030D0009B03332349F020919C0330919D03206191
:1030E00030939D0320939C03882349F080919C0397
:1030F00090919D03806290939D0380939C0380E058
:103100000F900F900F900F900F90DF91CF91089537
:10311000CF93DF9300D000D01F92CDB7DEB73A9A9D
:10312000429A84B1807F84B985B18F6085B987B1B7
:103130008C7F87B988B1836088B9CE0101960E94DF
:10314000771781E08093DF0189818F709A818F30BA
:1031500089F4892F8F70833069F48C818F7083306C
:1031600021F48D818F70833011F083E001C082E003
:103170008093DF0195FD03C083E08093DF010E940F
:10318000C21780E00F900F900F900F900F90DF917B
:10319000CF91089583ED91E00895CF93DF93CDB75C
:1031A000DEB7EF970FB6F894DEBF0FBECDBF80E657
:1031B0008BB98FEB8AB987EB9BE00197F1F700C0E1
:1031C00000004E9903C081E08093EB018091EB01F8
:1031D000811108C087E088B983EC87B915B88FEFF3
:1031E00084B905C017B88FEF88B914B885B90E94A3
:1031F000140E0E94AD0B0E94000A5C010E94AA0BF3
:10320000782E692E0E94F90D582E492E0E94CA1858
:103210008C018091EB01882329F0D801ED91FC917C
:103220000995580140E0BE016C5E7F4F80E090E060
:103230000E94900F20E030E040E050E0BE01695D68
:103240007F4FCE0144960E94840F8091EB01811143
:103250004AC00E943F0C99278130910541F00297A6
:1032600061F485E08093EA018CE291E03AC084E069
:103270008093EA0182E391E034C08091EB018823DE
:1032800091F00E94CA188C01DC011296ED91FC911C
:1032900013970995D8011696ED91FC911797CE01D9
:1032A0000196099520C00E94000A8C01DC0112964B
:1032B000ED91FC9113970995D8011696ED91FC912B
:1032C0001797CE01019609958981823029F4809360
:1032D000EA0186E291E005C083E08093EA0180E2A2
:1032E00091E00E947F0802E715E020E031E041E133
:1032F000BE01695D7F4F88E391E00E9428080E942B
:103300006F087894C12CD12CF12C812C912C312C6C
:10331000E12C00E010E083B78E6083BF83B781604B
:1033200083BF889583B78E7F83BF8091EC0188230C
:10333000E1F31092EC0189E89BE10197F1F700C0FD
:103340000000EE2021F091E0E916C9F154C010927E
:1033500079038091EB01811120C0AFEFCA1ADA0A1C
:10336000B9E7CB16D104CCF00E943F0C8130910517
:1033700049F0029781F4052D142DC12CD12C92E037
:10338000392E06C0072D162DC12CD12C3324339491
:10339000EE24E39402C0C12CD12CA114B10469F134
:1033A000D5011296ED91FC9113970995D5011696CA
:1033B000ED91FC911797CE01019609951EC0D80199
:1033C0001296ED91FC9113970995882341F0BFEF78
:1033D0008B1A9B0A8BE088169104A4F00CC0D801CC
:1033E0001696ED91FC911797CE0101960995FF2055
:1033F00039F0F39405C0E12C05C0FF24F39402C01A
:10340000812C912C0E947C08811129C08EEF0E9492
:103410007605823029F0833031F482E0282E04C012
:103420002224239401C0212C4F2DBE016C5E7F4FBE
:10343000CE0101960E94900FB2E0BF150CF4F12C62
:10344000222D30E0432D50E0BE01695D7F4FCE015B
:1034500044960E94840F61E1CE01879637C0809127
:10346000EA01298130E0482F082E000C550B241763
:10347000350709F050CF833021F14CF4823009F048
:103480004ACF8C819D8199AF88AF62E01DC08430A6
:1034900071F0853009F03FCF88E0FE013A96DE01F9
:1034A000D89601900D928A95E1F768E00DC08E8163
:1034B0009F81A885B98588AF99AFAAAFBBAF64E0FB
:1034C00003C08B8188AF61E0CE01C8960E942108BD
:1034D00022CF97FB072E16F4009407D077FD09D072
:1034E0000E94831A07FC05D03EF4909581959F4F6A
:1034F0000895709561957F4F0895EE0FFF1F059019
:10350000F491E02D0994AA1BBB1B51E107C0AA1F2F
:10351000BB1FA617B70710F0A61BB70B881F991F74
:103520005A95A9F780959095BC01CD010895FB01AE
:10353000DC0104C08D910190801921F4415050406C
:10354000C8F7881B990B0895FB01DC0102C00190AC
:103550000D9241505040D8F70895DC0101C06D93A1
:1035600041505040E0F70895DC01CB01FC01F9998E
:10357000FECF06C0F2BDE1BDF89A319600B40D92BF
:1035800041505040B8F70895DC01A40FB51F4150D9
:10359000504048F0CB01840F951F2E910E94D51A00
:1035A00041505040D0F70895262FF999FECF92BD93
:1035B00081BDF89A019700B4021639F01FBA20BDF8
:1035C0000FB6F894FA9AF99A0FBE0895F894FFCFBF
:1035D000E02080E02080E02080E0208000000000EB
:1035E000E02080E02080E02080E0208000000000DB
:1035F0000000A42052080000A42052100000A420C3
:1036000052470000A42052640000A4200101F109E7
:10361000C509BC09900900000000000104070B0F58
:1036200013171B1F252B32393F45494D505356590F
:103630005C5E6061626364000000000102030406D6
:10364000080A0C0E10121920262C343C3D3E3F4037
:103650004142434445464748494A00010203060C9B
:1036600012161F2832383C404345464748494A0015
:1036700000000000000000000000A60B850A7C0A84
:103680002F0A430A560A05F50DC70D850C7A0C0062
:1036900000EC0D455854454E4D4F54320003000088
:1036A0000000008818C2176E175A170000000002A9
:0A36B000455854454E4D4F5432006A
:00000001FF
